:100000000C9454050C94B5050C9456080C94B50545
:100010000C94B5050C94B5050C94B5050C94B50578
:100020000C94B5050C94B5050C94B6150C94B50557
:100030000C9465230C94B5050C94B5050C94B5058A
:100040000C94B5050C94B5050C94B5050C94B50548
:100050000C94B5050C94BA230C94B5050C94B50515
:100060000C94B5050C94B5050C94B5050C94B50528
:100070000C94B5050C94B5050C94B5050C94B50518
:100080000C94B5050C94B5050C94B5050C94B50508
:100090000C94B5050C94B5050C94B5050C94B505F8
:1000A0000C94B5050C94B5050C94B505D509D70984
:1000B000E309E309E309E309E309E309D909DB09F2
:1000C000DD09E309E309D709E509E309E3099F0924
:1000D000D509E309E309DB09E309E309E309E309D6
:1000E000E309E309DD09D509C109E309C509E30904
:1000F000E309E309A109D909E309E309CF09E30900
:10010000E309E309A309E109E309C309E309D709FD
:10011000E309E309D309C709E309C909DB09E309CD
:10012000E309E309D109CB09E309E309E309E30999
:10013000E309E309E309CD09E309A509E309E309B3
:10014000D909E309E309E109E309E309E309E3095B
:10015000E309E309E309E309E309A709E309E3097B
:10016000E309CF09E309E309E309E309E309E30943
:10017000E309E309E309E309A909E309AB09AD09C7
:10018000E309E309E309AF09B109B309E309B509D3
:10019000B709E309E309E309DF09B909E309BD097F
:1001A000BB09BF09E309E309E309E309E109090A16
:1001B000170A230A230AFB09230A230A230A230A0C
:1001C000230A230A230A230A230A230A230A230AC7
:1001D000230AFD09230AFF09230A230A230A230A03
:1001E0001B0A230A320A190A230A230A230A230AAA
:1001F000230A230A230A230A230A230A230A230A97
:10020000230AF3090F0A010A130A230A030A230A1D
:10021000070A230A110A050A150A0B0A0D0A230AFE
:10022000230A230A230A230A230A230AF509F709C2
:10023000F9091D0A1F0A230A230A230A210AAB0A05
:10024000C10ACF0ADD0AFD0A140B370B540BED0B64
:100250001A0CB10C0C0DF20C210D3C0D460D4D0D80
:10026000510D580D04142B1423152B14231577143A
:100270009A142315F11400157C197C19A619A619D6
:10028000011A2C1C2C1C2C1C351A2C1C201B201B6E
:10029000E61B2C1CFB1B191C007B46010203763A53
:1002A000687F6577482B353B6978796439141E3C43
:1002B0006A7A1D16041A1F3D6B061B070821203E93
:1002C0006C2C19091715223F6D11050B0A1C2340D0
:1002D0006E7E100D182425416F360E0C1227264213
:1002E0007037380F33132D43717534322F2E44720B
:1002F0007C7D28303174457351504A524D492A54FF
:1003000066594F5C5F4C4B4E62635A5D5E60295389
:1003100067585B56576147554842403E3C3A3B451B
:100320006843413F3D2B357E697A790078141E7C05
:100330006A7B1D16041A1F7F6B061B070821204DC0
:100340006C2C19091715224A6D11050B0A1C234C38
:100350006E49100D182425516F360E0C1227264FAA
:100360007037380F33132D52717534502F2E4E7253
:10037000397D283065314B735464586776012A778C
:100380003259745C5F66024662635A5D5E6029534F
:1003900044575B565561470380291E1F20212223A5
:1003A000242526272D2E2A2B141A0815171C180C65
:1003B00012132F302878041607090A0B0D0E0F337D
:1003C000343579311D1B06190511103637387D5526
:1003D0007A2C393A3B3C3D3E3F4041424353475FD4
:1003E0006061565C5D5E57595A5B626346483244B1
:1003F00045677B7F650301025250514F68696A6B04
:100400006C6D6E6F7071725800494C754A4D734B2C
:100410004E767C777E7466547225303258200062A6
:10042000253034582000772530325820002143539E
:10043000335F4630210A00214353335F46305F4526
:100440005252210A00214353335F46305F4F5652C8
:10045000210A00214353335F5245414459210A0088
:10046000214353335F455252210A00214353335FE6
:100470004F5652210A00214353325F45305F4630C8
:10048000210A00214353325F4630210A00214353A1
:10049000325F4530210A00214353325F494E4954AF
:1004A000210A00214353325F455252210A00214361
:1004B00053325F4F5652210A00214353315F45307A
:1004C0005F25303258210A00214353315F45525293
:1004D000210A00214353315F494E56210A004C2521
:1004E000752000532575200049443A25303458289A
:1004F0002564290A004D6F7573653A206E6F74206C
:10050000737570706F727465640A000A4552523ACE
:10051000253032580A0052257520005725752000D5
:10052000572575200057257520005825752000494E
:1005300025752000696E69740A000A4552523A25F1
:100540003032580A000A4B6579626F617264207319
:10055000746172742E0A000A55534220636F6E66EE
:100560006967757265642E0A000A0A544D4B3A6237
:10057000366363626163642B2F4C5546410A0A005F
:100580003403490042004D00200050004300200089
:100590006B006500790062006F006100720064000A
:1005A000200063006F006E0076006500720074002A
:1005B0006500720000000E0374002E006D002E0016
:1005C0006B002E00000004030904090274000401FA
:1005D00000A03209040000010301010009211101FA
:1005E00000012240000705810308000A09040100F8
:1005F0000103000000092111010001223600070556
:10060000820308000A090402000203000000092115
:1006100011010001222200070583032000010705C4
:100620000303200001090403000103000000092165
:100630001101000122390007058403200001120185
:10064000100100000008EDFEEE1B01000102000198
:1006500005010906A101050719E029E71500250193
:10066000950875018102050819012905950575018F
:1006700091029501750391010507190029F71500ED
:10068000250195F875018102C00631FF0974A101A9
:100690000975150026FF0095207508810209761559
:1006A0000026FF00952075089102C005010980A170
:1006B0000185021601002637001A81002AB700754D
:1006C0001095018100C0050C0901A10185031601E7
:1006D00000269C021A01002A9C02751095018100D7
:1006E000C005010906A101050719E029E715002544
:1006F00001950875018102950175088101050819A8
:100700000129059505750191029501750391010572
:1007100007190029FF150026FF00950675088100BE
:10072000C0636F6E73756D65723A20253034580A58
:100730000073797374656D3A20253034580A000AC5
:10074000002530325820006B6579626F6172643A1F
:1007500020004C45443A20253032580A00253032DA
:10076000583A202530386225730A00722F632030F2
:10077000313233343536370A0064656C5F6B657926
:100780005F6269743A2063616E27742064656C3A15
:1007900020253032580A006164645F6B65795F62BE
:1007A00069743A2063616E2774206164643A20257D
:1007B0003032580A003F00433E20004C25640A00B6
:1007C0000A092D20436F6E736F6C65202D0A455307
:1007D000432F713A09717569740A000A092D204D79
:1007E00061676963202D0A643A0964656275670A66
:1007F000783A096465627567206D61747269780A78
:100800006B3A096465627567206B6579626F617226
:10081000640A6D3A096465627567206D6F7573656A
:100820000A763A0976657273696F6E0A733A0973CC
:1008300074617475730A633A09636F6E736F6C65E4
:10084000206D6F64650A302D343A096C61796572E8
:10085000302D34284631302D4634290A50617573C5
:100860003A09626F6F746C6F616465720A6E3A095F
:100870004E4B524F0A003F004E4B524F3A206F668C
:10088000660A004E4B524F3A206F6E0A0074696D33
:1008900065725F72656164333228293A20253034ED
:1008A0006C580A006B6579626F6172645F6E6B727F
:1008B0006F3A2025580A006B6579626F6172645F38
:1008C00069646C653A2025580A006B6579626F612E
:1008D00072645F70726F746F636F6C3A2025580A90
:1008E00000686F73745F6B6579626F6172645F6CCF
:1008F00065647328293A2025580A000A092D2053D7
:100900007461747573202D0A004743433A20352ED5
:10091000342E30204156522D4C4942433A20322E3B
:10092000302E30204156525F415243483A20617682
:1009300072350A004F5054494F4E533A204C554699
:10094000412045585452414B455920434F4E534F37
:100950004C4520434F4D4D414E44204E4B524F206D
:100960004B45594D41505F53454354494F4E2042EA
:100970004F4F544C4F414445525F53495A450A002A
:100980004255494C443A2062366363626163642B8A
:10099000202831323A32373A3533204170722032D2
:1009A000382032303230290A005649443A20307813
:1009B0004645454428742E6D2E6B2E2920504944FF
:1009C0003A203078316265652849424D20504320F5
:1009D0006B6579626F61726420636F6E76657274A5
:1009E000657229205645523A203078303030310A2D
:1009F00000444553433A20636F6E76657274204914
:100A0000424D205043206B6579626F61726420749F
:100A10006F205553420A000A092D205665727369EA
:100A20006F6E202D0A000A6D6F7573653A206F6630
:100A3000660A000A6D6F7573653A206F6E0A000AC8
:100A40006B6579626F6172643A206F66660A000AAC
:100A50006B6579626F6172643A206F6E0A000A6D8D
:100A600061747269783A206F66660A000A6D617473
:100A70007269783A206F6E0A000A64656275673A97
:100A8000206F6E0A000A64656275673A206F6666B9
:100A90000A000A0A626F6F746C6F616465722E2EB1
:100AA0002E2000433E20000011241FBECFEFDAE0CD
:100AB000DEBFCDBF04B603FE41C080918503909197
:100AC0008603A0918703B09188038730904BA7409D
:100AD000B04BA1F510928503109286031092870304
:100AE0001092880314BE0FB6F894A8958091600008
:100AF000886180936000109260000FBE1092010820
:100B000010920008E3E0F0E089E080935700E49160
:100B1000E695E370E150E33040F4F0E0EE0FFF1FA4
:100B2000E35DFE4F8081918102C080E090E1E0E0D2
:100B3000F0E8E81BF90BF695E795099511E0A0E0C0
:100B4000B1E0ECE7FBE402C005900D92A433B107DD
:100B5000D9F723E0A4E3B1E001C01D92A538B207A4
:100B6000E1F70E9419110C94BC250C940000FF932E
:100B7000EF93E0913401F0913501309709F0099538
:100B8000EF91FF910895FC018591803011F0EFDF26
:100B9000FBCF0895FF27E0E230E247FF0CC041950C
:100BA00097FF09C0EDE26095709580959095611D65
:100BB000711D811D911D27FF02C0219530E350E278
:100BC000AA27660F771F881F991FAA1FA41710F066
:100BD000A41B63955A95A9F7AA3008F0A95FA05DF8
:100BE000AF93F395611571058105910541F7ED32DC
:100BF00011F4EF93F395F21718F43F93F395FBCFAD
:100C00008F91B5DFFA95E1F70895E991F991859112
:100C1000803021F0853219F0AADFF9CF089520E065
:100C2000E89455915532C1F3503311F468945591BD
:100C30005A3348F4505390F3220F022E220F220F02
:100C4000200D250FF4CF0EF42195899199915336FB
:100C500019F3533729F1533559F1BC0188279927E6
:100C6000E8945C3621F489919991689455915436B1
:100C700039F446EF7EF077FF0DC08FEF9FEF0AC08B
:100C800055374AE039F0583540E121F0523642E01C
:100C900009F00895FF93EF937DDFEF91FF91B7CFB8
:100CA000FF93EF93FC0181918030B9F360DFFBCFBC
:100CB000FF93EF9368DFF1CFDF93CF93CDB7DEB72C
:100CC0002596A3DFCF91DF910895282F80913F01D2
:100CD000823071F08330B1F0813001F5E62FF0E021
:100CE00038E0739FE00DF11D1124E856FC4F13C04E
:100CF000E62FF0E088E0789FE00DF11D1124E85E1A
:100D0000FC4F09C0E62FF0E038E0739FE00DF11DC5
:100D10001124E856FD4FE491E03819F480E090E0AA
:100D200008959E2F9077892F90E034E095958795D0
:100D30003A95E1F738E0239F800D911D112444E09E
:100D4000880F991F4A95E1F7EF709C012E0F311D16
:100D5000F901EE0FFF1FE050F84985919491089535
:100D60005998519A08955198599A08955898509AB7
:100D700008955098589A08955198599A85E08A95FF
:100D8000F1F7000089B18695817008955098589ABE
:100D900085E08A95F1F7000089B181700895CF93BD
:100DA000DF93EC010E94BC06882341F0209731F0CC
:100DB00085E08A95F1F700002197F4CFCE01DF910D
:100DC000CF910895CF93DF93C2E3D0E00E94BC0699
:100DD000811108C0209731F085E08A95F1F7000075
:100DE0002197F4CFCE01DF91CF9108952E982698C8
:100DF0002F9827980E94B0060E94B906E9E6F0E015
:100E0000808188608083E9980895E19AE99A0E9438
:100E1000B3060C94B906E9980E94B0060C94B90682
:100E2000CF932FB7F8948091020190910301AC0108
:100E3000442741155F4F21F0C92FAC015F6F07C0F8
:100E40008F3F4FEF940741F0C82F4FEF5FEF509364
:100E500003014093020101C0CFEF2FBF9C012F6F10
:100E60002F3F3F4F81F02091720320FF1FC09F93BF
:100E70008F938FE194E09F938F930E945C060F9075
:100E80000F900F900F90CF3F99F08091720380FFE9
:100E900012C01F92CF9388E194E09F938F930E949A
:100EA0005C060F900F900F900F9005C0CF3F19F484
:100EB0008FEF9FEF02C08C2F90E0CF910895CF93DA
:100EC000CAE1C15069F00E9410078F3F2FEF9207CF
:100ED00049F48FE99FE00197F1F700C00000F1CFDE
:100EE0008FEF9FEFCF91089580E090E890930101FC
:100EF000809300018FEF9FEF909303018093020195
:100F00000895EF92FF920F931F93CF93DF93082FD3
:100F1000109237018091720380FF0CC01F920F93D3
:100F200086E294E09F938F930E945C060F900F904F
:100F30000F900F90E9980E94B0060E94B9068FE8C2
:100F400091E00197F1F700C000000E94B6060E94F0
:100F5000B30680E197E20E94CF06892B11F481E06D
:100F600079C0C0E0D0E0FF24F39410E0EE24E394D5
:100F700090E59A95F1F7C8010C2E02C095958795DA
:100F80000A94E2F780FF04C0FE240E94B90602C062
:100F90000E94B6060E94E206892B11F482E05AC034
:100FA00082E390E00E94CF06892B11F483E052C0C7
:100FB0002196C830D105E1F680E58A95F1F7FF204A
:100FC00019F00E94B90602C00E94B6060E94E2060D
:100FD000892B11F484E03EC082E390E00E94CF06AA
:100FE000892B11F485E036C090E59A95F1F70E94BF
:100FF000B906C2E3D0E00E94C606882341F02097DC
:1010000041F025E02A95F1F700002197F4CFCD2B90
:1010100011F486E01FC082E390E00E94CF06892B86
:1010200011F487E017C00E94E206892B19F0C2E391
:10103000D0E009C088E00EC0209759F085E08A957D
:10104000F1F7000021970E94C6068823A9F3CD2B53
:10105000B9F489E0809337018091370180618093F2
:1010600037010E94B3060E94B906E19AE99A8FEF10
:101070009FEFDF91CF911F910F91FF90EF90089517
:101080008FEF9FEF90930301809302010E947407FA
:101090000E94B3060E94B906E19AE99ADF91CF91C6
:1010A0001F910F91FF90EF900C945F071F920F928A
:1010B0000FB60F9211242F933F934F935F938F930B
:1010C0009F9329B121708091730340910001509149
:1010D00001014115504819F48093360112C09091D6
:1010E0003601891771F09F5F891759F090E290934C
:1010F00037018093360180E090E89093010180935E
:10110000000180910001909101019695879590933F
:10111000010180930001222349F080910001909108
:10112000010190689093010180930001809100017A
:101130009091010199278035910509F455C090F4EB
:101140008031910509F450C020F4892B09F4A0C026
:1011500067C08032910509F49BC08034910509F481
:1011600097C05EC0803A910581F040F480389105C7
:1011700009F48EC080399105B9F152C0803C9105C7
:1011800031F0803D910581F14BC084E613C0809120
:10119000000190910101892F99279093010180937B
:1011A000000183E02FC0882379F025E02A95F1F72C
:1011B00000008150499BF7CF07C0882349F095E094
:1011C0009A95F1F7000081504999F7CF811160C0DD
:1011D0008091000190910101892F9927909301013D
:1011E0008093000182E00EC0809100019091010186
:1011F00036E0969587953A95E1F7909301018093B3
:10120000000181E0809338018091000190910101FB
:1012100099278F3F9105A1F48FEF8093370110C07C
:1012200080E88093370180E090E8909301018093FB
:10123000000180E09FEF909303018093020128C09A
:101240008091020190910301882781159F4F19F029
:1012500080E4809337018091020190910301982FDF
:10126000882790930301809302012091000130911F
:1012700001018091020190910301822B909303015F
:101280008093020180E090E8909301018093000137
:101290009F918F915F914F913F912F910F900FBE32
:1012A0000F901F901895CF93C82F8DEE0E94810745
:1012B0008C2FCF910C948107E82FE695E695E69563
:1012C000EF70F0E0EE5BFE4F4081282F277081E049
:1012D00090E002C0880F991F2A95E2F7242F30E092
:1012E00028233923232B11F4842B80830895E82F9E
:1012F000E695E695E695EF70F0E0EE5BFE4F208117
:10130000382F377081E090E002C0880F991F3A951E
:10131000E2F7422F50E048235923452B19F08095DE
:10132000822380830895482F50E0FA013397E138F3
:10133000F10508F048C0EA5AFF4F0C94B62587E142
:1013400008958FE108958CE5089580E6089582E67A
:10135000089587E2089583E508958FE2089589E36B
:10136000089587E308958FE3089587E408958FE44F
:10137000089586E508958EE508958FE6089580E046
:10138000089585E608958EE608958FE7089580E331
:10139000089588E3089580E4089588E4089580E539
:1013A000089587E508958FE5089588E1089588E018
:1013B000089580E2089580E1089589E108958DE619
:1013C000089588E208958F7708958FE00895CF9368
:1013D000482F50E0FA017C97E834F105A0F5E95276
:1013E000FF4F0C94B62585E53EC08AE53CC08BE5F1
:1013F0003AC08CE538C08DE536C08EE534C08FE547
:1014000032C080E630C081E62EC082E62CC083E682
:101410002AC08FE628C081E726C082E724C084E77F
:1014200022C085E720C087E71EC088E71CC08AE786
:101430001AC08CE718C08FE716C080E714C089E790
:1014400012C08BE710C0C82F1F928F9389EB94E0D6
:101450009F938F930E945C060F900F900F900F90B8
:101460008C2F01C084E5CF9108950F931F93CF93E4
:10147000DF930E9493238C010E941007EC010196D8
:1014800031F4C8010E94AB23843F9140A8F3CE0100
:10149000DF91CF911F910F9108950E94F6060C9451
:1014A000050780917203816080937203E2E4F1E0AA
:1014B000119281E0E235F807D9F70895E82FF0E0BE
:1014C000EE5BFE4F80810895E2E4F1E0119281E04D
:1014D000E235F807D9F70895982F82FB882780F91D
:1014E00090FD826091FD84600C945309CF93DF934B
:1014F00080913701882311F1809137011F928F93DA
:101500008AE395E09F938F930E945C068091370158
:1015100080750F900F900F900F9071F480913E01A5
:10152000893051F484E395E09F938F930E945C0689
:1015300010923E010F900F9010923701E0913E0102
:101540008E2F90E08A30910508F0B1C3FC01E15E76
:10155000FE4F0C94B6250E9493239F938F938FE2A6
:1015600095E09F938F930E945C0610923F0110922A
:101570004101109240010E94640A0E942C1981E0EE
:1015800035C00E940B072E98269A2F98279A0E9402
:10159000932390933D0180933C0182E00BC08091A6
:1015A0003C0190913D010E94AB23853F914008F49E
:1015B0007EC383E080933E017AC32E9826982F98AD
:1015C00027980E9474070E9405070E9493239F9307
:1015D0008F938AE295E09F938F930E945C060E940E
:1015E000932390933D0180933C0184E080933E01DE
:1015F0000F900F900F900F905AC30E941007019602
:1016000009F455C30E9493239F938F9385E295E03D
:101610009F938F930E945C060E94932390933D01B9
:1016200080933C0185E0E2CF80913C0190913D01A7
:101630000E94AB23853F914018F087E080933E01E4
:101640000E941007019609F432C30E9493239F93CE
:101650008F9380E295E09F938F930E945C060E9497
:10166000932390933D0180933C0186E0BFCF80910E
:101670003C0190913D010E94AB23853F914018F0C1
:1016800087E080933E010E941007019609F40FC382
:101690000E9493239F938F938BE195E09F938F9369
:1016A0000E945C0687E0A2CF0E9493239F938F93B2
:1016B00086E195E09F938F930E945C0682EF0E94E3
:1016C00081070F900F900F900F908F3F2FEF920791
:1016D00089F08A3F910589F40E94350A8F3F3FEFD8
:1016E000930771F0D82FCC270E94350A9E01282B32
:1016F000C90108C08FEF9FEF05C08EEF9FEF02C0BA
:1017000080E090E090934101809340018091370107
:10171000882381F0809137011F928F938BE095E0B1
:101720009F938F930E945C06109237010F900F9049
:101730000F900F908091400190914101009711F41A
:1017400082E029C08F3F3FEF930711F481E023C06F
:101750008E3F2FEF9207A1F38F3F910559F485EF4C
:1017600094E09F938F930E945C0610923F010F902C
:101770000F9019C086383BEA930781F480EF0E94EE
:1017800081078A3F9105E1F683E00E9481078A3F45
:101790009105B1F683E080933F0105C0882781154C
:1017A0009F4BC1F3CDCF80913F011F928F938091CA
:1017B00041018F93809140018F9388EE94E09F9335
:1017C0008F930E945C0688E080933E010F900F90FB
:1017D0000F900F900F900F906AC20E9493239F93D7
:1017E0008F9383EE94E09F938F930E945C060F90FB
:1017F0000F900F900F9080913F01823031F0833035
:1018000041F488EF0E94810704C00E94A4160E9440
:101810006C0A89E080933E010E9493239F938F93EB
:101820008EED94E09F938F930E945C060F900F9033
:101830000F900F90C0913F01C23009F47EC0C330B9
:1018400009F43FC1C13009F032C20E9410078F3F36
:101850003FEF930709F42BC29C012F7733272236E1
:10186000310548F083ED94E09F938F930E945C06CE
:1018700010923B01FEC020913B01223009F444C08C
:1018800028F4222351F0213019F154C0233009F4F7
:1018900047C0243009F449C04DC0803E910569F02D
:1018A0001CF4009739F00EC0813E910549F08F3F3E
:1018B000910541F488EC94E0D8C0C0933B01F7C196
:1018C00082E02BC08038910508F45BC18F77A9C1F5
:1018D0008633910579F124F48A32910539F42AC0CE
:1018E0008A3A910539F1863B910521F180389105BD
:1018F00028F40E94E7090E945C091CC08F770E94AF
:10190000E7090E94770916C08D31910529F08D39BC
:10191000910581F484E001C083E080933B01C7C15D
:101920008534910539F485E52CC18534910511F490
:1019300085E577C110923B01BAC10E9410078F3F25
:101940002FEF920709F4B3C1E0913A014E2F50E016
:101950004930510508F0B2C0FA01E75DFE4F0C9422
:10196000B625803E910569F18CF48338910569F1C3
:101970002CF4009771F58EEA94E0E8C08438910564
:1019800031F18A3A910509F490C123C0803F910555
:10199000D1F02CF4813E9105E1F484E086C08C3FC7
:1019A000910509F482C18F3F910599F40E94640A60
:1019B00083EA94E09F938F930E945C0610923A0111
:1019C00058C082E072C081E070C082E063C08FE6E0
:1019D00061C08038910508F4D4C00E94640A87E988
:1019E00094E043C08935910509F468C0803F9105B2
:1019F00021F08231910519F461C083E056C0109244
:101A00003A018038910518F40E949309BAC00E94E7
:101A1000640A8DE894E029C08338910529F0843860
:101A2000910521F48FE648C082E046C010923A0149
:101A30008038910508F4F5C00E94640A83E894E0B8
:101A400014C010923A018231910509F430C18935F0
:101A5000910509F42CC18038910518F40E9493096E
:101A6000E0C00E94640A86E794E09F938F930E94EF
:101A70005C060F900F9019C18431910529F0803FC9
:101A80009105E1F486E011C085E00FC0873791052C
:101A9000A9F480E00E945C0911C0449779F487E0C2
:101AA00004C0803F910551F488E080933A01FFC063
:101AB0008737910519F480E00E94770910923A0166
:101AC000F6C00E9410078F3F3FEF930709F4EFC065
:101AD00020913901213009F45AC038F0223009F43C
:101AE000ACC0233009F4CCC0E2C08638910509F4BB
:101AF0003FC09CF483389105B9F13CF4009721F183
:101B000080389105D9F582E0B3C08438910571F130
:101B10008538910599F58BE034C08C38910561F1D9
:101B200044F48738910531F18B38910539F581E01E
:101B300028C0803F9105B1F08F3F910581F08D382D
:101B40009105E1F48AE01DC08BE694E09F938F93AA
:101B50000E945C060E94640A0E942C196BC080E6F9
:101B600094E083CF81E084C082E00BC08FE709C09E
:101B700086E007C080E005C089E003C08038910599
:101B800018F40E945C0993C083E594E04FC0863846
:101B90009105E1F1DCF483389105A1F17CF4009723
:101BA000D9F585E494E09F938F930E945C060E9490
:101BB000640A0E942C19109239013CC084389105A6
:101BC00019F18538910541F58BE06CC08C38910591
:101BD000F9F04CF48738910509F463C08B3891050E
:101BE000D9F481E05FC08D389105A1F08F3F910558
:101BF00099F487E394E09F938F930E945C06109280
:101C0000390137CF82E04EC08FE74CC086E04AC032
:101C100089E048C08AE046C01092390180389105B9
:101C200018F40E94770943C08DE294E09F938F934C
:101C30000E945C060F900F903AC08532910591F09A
:101C40003CF48631910581F04E97A9F480E00DC0F7
:101C50008632910529F0803F910569F483E008C040
:101C60008DE503C083E501C081E50E945C0905C0E4
:101C7000809339011CC00E94640A1092390117C078
:101C80008E31910571F024F44697A9F781E50AC0D9
:101C90008532910521F0869771F78DE503C083E5C4
:101CA00001C080E00E947709E8CF10923E0181E0F8
:101CB000DF91CF9108958091760208950895CF9392
:101CC000DF9300D01F92CDB7DEB720917C03243084
:101CD00021F523E029839B838A8382E08093E900B6
:101CE0008FEF9091E800815095FD06C095ED9A9593
:101CF000F1F700008111F5CF8091E80085FF0DC05C
:101D000040E050E063E070E0CE0101960E94CF1207
:101D10008091E8008E778093E8000F900F900F90ED
:101D2000DF91CF910895CF93DF9300D01F92CDB76D
:101D3000DEB720917C03243029F522E029838058E6
:101D400091099B838A832093E9008FEF9091E800AB
:101D5000815095FD06C095ED9A95F1F7000081112F
:101D6000F5CF8091E80085FF0DC040E050E063E0D2
:101D700070E0CE0101960E94CF128091E8008E772C
:101D80008093E8000F900F900F90DF91CF9108950E
:101D9000CF93DF93EC0190917C03943009F048C01D
:101DA000809114018823D9F0809115018823B9F01E
:101DB0009093E90081E8815049F09091E80095FD09
:101DC00005C09AE29A95F1F700C0F5CF8091E8003E
:101DD00085FF2EC040E050E060E270E019C081E075
:101DE0008093E90081E8815059F09091E80095FDD9
:101DF00007C0EFE3F1E03197F1F700C00000F3CF47
:101E00008091E80085FF14C040E050E068E070E099
:101E1000CE010E94CF128091E8008E778093E80077
:101E200080E2FE01A6E5B2E001900D928A95E1F70D
:101E3000DF91CF910895CF93C0915401C1110BC090
:101E40000E949F23643C79408105910520F081E048
:101E500080935401C1E08C2FCF910895FF920F938E
:101E60001F93CF93DF93D82F0FB607FE83C08091C7
:101E70007C03843081F08091070190E001962091ED
:101E8000090130E0822393232091080130E082177A
:101E9000930709F0CDC00E941B0F811110C08091E3
:101EA000070190E001962091090130E082239323FD
:101EB0002091080130E08217930709F0B9C00E9411
:101EC00093238C01C091E900CF709091EC00892F91
:101ED000817090FD80E8C82B83E08093E90085E065
:101EE000F82E8091EB0085FD42C08091EB0080FFD1
:101EF0003EC08091EE0087FF3AC08091080190912A
:101F00000701981709F457C09091E80095FF8EC01B
:101F1000E0910501F0910601E80FF11D20818F5F2E
:101F2000909109018923809308012093F100809109
:101F3000E80085FDE2CF8091E80080FFDECF809150
:101F4000E8008E778093E800F0920401D6CF80916C
:101F5000070190E001962091090130E0822393234C
:101F60002091080130E08217930709F44CC0CF702C
:101F7000C093E90040910701842F90E001962091E1
:101F8000090130E0822393232091080130E0821779
:101F9000930709F450C0E0910501F0910601E40FA8
:101FA000F11DD083809107018F5F909109018923F2
:101FB0008093070140C08091E80085FF37C0D0932F
:101FC000F10021E03091F3008091F20090E0932B3A
:101FD000892B91F08091E80080FF0EC08091E8008D
:101FE00085FF03C01092F100F9CF8091E8008E7751
:101FF0008093E800F0920401222309F4A8CFCF7067
:10200000C093E90018C080910401882309F4AFCF80
:102010000E9493239C018017910711F4890161CFDD
:1020200090910401915090930401F8CF20E0CACF21
:1020300040910701B0CF80E0DF91CF911F910F91C8
:10204000FF90089580917B03811104C00E943B158D
:102050000C949815089510927B030895089542E01A
:1020600061EC81E00E94481242E061EC82E00E9453
:10207000481242E261EC83E00E94481242E261ECC5
:1020800084E00C94481280917E03833009F455C09B
:1020900030F4813071F0823009F48EC008958A30B6
:1020A00009F47AC08B3009F460C0893009F09CC013
:1020B00020C080917D03813A09F096C08091E800AC
:1020C000877F8093E8008091810390918203892B20
:1020D00021F460E286E592E003C060E080E090E0F9
:1020E00070E00E941C138091E8008B778093E800D9
:1020F000089580917D03813209F076C0809181033B
:1021000090918203009719F0039709F06DC08091B8
:10211000E800877F8093E8008091E80082FD05C099
:1021200080917C038111F8CF5FC08091F100809392
:1021300076028091E8008B7753C080917D03813ACD
:1021400009F052C08091810390918203892B09F09C
:102150004BC08091E800877F8093E8008091E80081
:1021600080FFFCCF8091140136C080917D038132C5
:10217000D9F58091810390918203892BA9F58091F3
:10218000E800877F8093E8000E947D1280917F03A2
:10219000809314010C942C1980917D03813221F5D8
:1021A0008091E800877F8093E8000E947D128091F3
:1021B000800380937702089580917D03813AA1F492
:1021C0008091E800877F8093E8008091E80080FF9D
:1021D000FCCF809177028093F1008091E8008E77A8
:1021E0008093E8000C947D1208958091760280938C
:1021F0005501109276020E94640A0C942C190C94DA
:10220000F5100E94402380917A03882329F00E94D0
:102210004D2381110C94321208950E946123809104
:1022200055018093760208950C940D1108950C9435
:102230001611CF9384B7877F84BF0FB6F894A89503
:1022400080916000886180936000109260000FBEF2
:1022500090E080E80FB6F89480936100909361005D
:102260000FBE8EE29FE00E9413238AE091E00E945D
:102270009F1689E695E00E94C3050E944D0A0E94C0
:1022800053170E943B150E94981578940E94551789
:1022900080917C03843029F00E9484160E941611DC
:1022A000F7CF87E595E00E94C3050E94171185E4EA
:1022B00095E00E94C305C3E080917C03853019F44A
:1022C0000E940111F9CF0E9459172091E40030912A
:1022D000E50080915201909153012817390709F4C4
:1022E00068C08091E4009091E50090935301809341
:1022F00052010E941B0F882309F45BC080917C036C
:10230000843009F056C08091E9008F702091EC0074
:10231000922F917020FD90E8892BC093E900909155
:10232000EB0090FF43C09091EE0097FF3FC090916B
:10233000080120910701291709F12091E80025FFE4
:102340001DC0E0910501F0910601E90FF11D3081FA
:102350009F5F209109019223909308013093F1002F
:102360009091E80095FDE3CF9091E80090FFDFCFDA
:102370009091E8009E779093E800D9CF9091F30078
:102380002091F20030E0392B232B81F09091E8006E
:1023900090FF0CC09091E80095FF03C01092F100EF
:1023A000F9CF9091E8009E779093E8008F7080932A
:1023B000E9000E94841680CF292F3327233031056E
:1023C000C9F060F42130310581F02230310509F087
:1023D00041C084E790E02AEC35E040C0213231056D
:1023E000E1F02232310531F135C082E190E02EE397
:1023F00036E034C099278130910549F028F00297E2
:1024000049F5E0E8F5E005C0E6ECF5E002C0E6EBF2
:10241000F5E0849190E09F0121C064307105D0F413
:10242000660F771FFB01EC5DFE4F2081318189E053
:1024300090E014C06430710568F4FB01EE0FFF1FDB
:10244000E45EFE4F20813181FB01E85EFE4F80811A
:1024500090E004C080E090E020E030E0FA013183B9
:102460002083089580E189BD82E189BD09B400FE21
:10247000FDCF8091D8008F7D8093D8008091E000BF
:1024800082608093E0008091E00081FDFCCF0895A0
:10249000982F973068F59093E900981739F070916C
:1024A000EC002091ED005091F00003C0242F762F16
:1024B00050E021FD02C09F5FECCF3091EB003E7FEA
:1024C0003093EB003091ED003D7F3093ED00309183
:1024D000EB0031603093EB007093EC002093ED0043
:1024E0005093F0002091EE0027FDE5CF80E00895A5
:1024F0008F708093E90081E0089580917D0387FFCC
:1025000011C08091E80082FD05C080917C0381119B
:10251000F8CF11C08091E8008B770BC080917C03CD
:10252000882349F08091E80080FFF8CF8091E8008F
:102530008E778093E80008952091E4003091E500C3
:1025400095E64091EC00842F817040FF23C080917C
:10255000E80080FD1DC080917C03882399F08530C0
:1025600099F08091EB0085FD11C04091E4005091FD
:10257000E5002417350729F3915011F09A01E1CFB6
:1025800084E0089582E0089583E0089581E008954D
:1025900080E008954091E80042FFDDCF0895CF929A
:1025A000DF92EF92FF920F931F93CF93DF93EC0193
:1025B0008B017A010E949C12811135C0E114F10453
:1025C00039F0F70180819181081B190BC80FD91FC1
:1025D000C12CD12C0115110529F18091E80085FD50
:1025E00018C08091E8008E778093E8000E948416DE
:1025F000E114F10449F0F70180819181C80ED91EE0
:10260000D182C08285E00FC00E949C12882311F302
:102610000AC089918093F10001501109FFEFCF1A90
:10262000DF0AD8CF80E0DF91CF911F910F91FF900B
:10263000EF90DF90CF900895209183033091840331
:102640002617370748F06115710539F42091E80025
:102650002E772093E80001C0B901FC0120E061154C
:10266000710579F180917C038823F1F18530F1F1D6
:102670008091E80083FD3CC08091E80082FD2EC07F
:102680008091E80080FFEBCF2091F3008091F20071
:1026900090E0922B6115710551F08830910538F466
:1026A00021912093F100615071090196F3CF21E04F
:1026B000089709F020E08091E8008E778093E80089
:1026C000CECF2111CFCF0AC080917C03882361F047
:1026D000853061F08091E80083FD0AC08091E800B8
:1026E00082FFF2CF80E0089582E0089583E00895AC
:1026F00081E00895209183033091840326173707E2
:1027000048F06115710539F42091E8002E77209387
:10271000E80001C0B901FC0120E06115710591F1EB
:1027200080917C03882309F440C0853009F43FC0C0
:102730008091E80083FD3DC08091E80082FD2FC0BC
:102740008091E80080FFE9CF2091F3008091F200B2
:1027500090E0922B6115710559F08830910540F495
:1027600024912093F1003196615071090196F2CFC6
:1027700021E0089709F020E08091E8008E778093AF
:10278000E800CBCF2111CCCF0AC080917C038823F5
:1027900061F0853061F08091E80083FD0AC080918E
:1027A000E80082FFF2CF80E0089582E0089583E0A0
:1027B000089581E008951F93CF93DF93CDB7DEB7DF
:1027C000AA970FB6F894DEBF0FBECDBFEDE7F3E0DA
:1027D0008091F100819323E0E538F207C9F70E9468
:1027E00043108091E80083FF2EC180917D0390917A
:1027F0007E03492F50E04A30510508F024C1FA0108
:10280000EE5CFE4F0C94B625803821F0823809F03A
:102810001AC108C08091790390917A03992389F0B5
:1028200082600FC0809181038F70873008F00BC1E8
:102830008093E9008091EB0085FB882780F9109256
:10284000E9009091E800977F9093E8008093F10071
:102850001092F100D1C0282F2D7F09F0F4C08823F9
:1028600019F0823061F0EFC080917F03813009F070
:10287000EAC0933009F080E080937A032EC0809103
:102880007F0381112AC0809181038F702FEF280F61
:10289000263008F0D8C08093E9002091EB0020FF9B
:1028A0001CC0933021F48091EB00806214C09091A1
:1028B000EB0090619093EB0021E030E0A90102C0B1
:1028C000440F551F8A95E2F74093EA001092EA0000
:1028D0008091EB0088608093EB001092E90080917A
:1028E000E800877F8093E8000E947D12ACC08111D0
:1028F000AAC010917F031F778091E3008078812B1D
:102900008093E3008091E800877F8093E8000E9435
:102910007D128091E80080FFFCCF8091E300806809
:102920008093E300111102C082E001C083E0809334
:102930007C0389C08058823008F085C080917F0375
:10294000909180038C3D53E0950779F583E08A836D
:102950008AE289834FB7F894DE01139620E03EE0C7
:1029600051E2E32FF0E050935700E49120FF03C0C1
:10297000E295EF703F5FEF708E2F90E0EA3010F03D
:10298000C79601C0C0968D939D932F5F243149F760
:102990004FBF8091E800877F8093E8006AE270E093
:1029A000CE0101960E941C1316C0609181037091A4
:1029B0008203AE014F5F5F4F0E94DC11BC01892B87
:1029C00009F441C09091E800977F9093E8008981D5
:1029D0009A810E947A138091E8008B778093E800B7
:1029E00032C0803881F58091E800877F8093E800CD
:1029F000809178038093F1008091E8008E7772CF08
:102A0000811121C080917F039091800399270297C3
:102A1000D4F48091E800877F8093E80080917F0361
:102A2000809378030E947D1280917803811106C003
:102A30008091E30087FD02C081E001C084E08093C3
:102A40007C030E942F108091E80083FF0AC08091D0
:102A5000E800877F8093E8008091EB00806280939C
:102A6000EB00AA960FB6F894DEBF0FBECDBFDF9184
:102A7000CF911F9108950E94A9150E94B115E0EE13
:102A8000F0E0808181608083E8EDF0E080818F77E5
:102A9000808319BCA7EDB0E08C918E7F8C938081F0
:102AA0008F7E808310927B0308950F931F93CF93A3
:102AB000DF930E94A9150E94B115C8EDD0E088816E
:102AC0008F77888388818068888388818F7D8883D9
:102AD00019BC10927C031092780310927A03109222
:102AE000790300EE10E0F80180818B7F808388817C
:102AF0008160888342E060E080E00E944812E1EE5D
:102B0000F0E080818E7F8083E2EEF0E08081816062
:102B10008083808188608083F80180818E7F8083BC
:102B2000888180618883DF91CF911F910F910895F3
:102B3000E8EDF0E080818F7E8083E7EDF0E080813A
:102B40008160808384E082BF81E080937B030C946A
:102B50005515E8EDF0E080818E7F80831092E200D1
:102B600008951092DA001092E10008951F920F92DA
:102B70000FB60F9211242F933F934F935F936F9350
:102B80007F938F939F93AF93BF93EF93FF93809126
:102B9000E10082FF0BC08091E20082FF07C08091BC
:102BA000E1008B7F8093E1000E9483168091DA0020
:102BB00080FF1FC08091D80080FF1BC08091DA0089
:102BC0008E7F8093DA008091D90080FF0DC080E174
:102BD00089BD82E189BD09B400FEFDCF81E080930B
:102BE0007C030E94221005C019BC10927C030E9435
:102BF0002B108091E10080FF19C08091E20080FFDE
:102C000015C08091E2008E7F8093E2008091E20007
:102C100080618093E2008091D80080628093D80028
:102C200019BC85E080937C030E94FF108091E10035
:102C300084FF30C08091E20084FF2CC080E189BD18
:102C400082E189BD09B400FEFDCF8091D8008F7D5F
:102C50008093D8008091E1008F7E8093E100809185
:102C6000E2008F7E8093E2008091E2008160809399
:102C7000E20080917803882311F084E007C08091FE
:102C8000E30087FD02C081E001C083E080937C0304
:102C90000E9414118091E10083FF24C08091E20022
:102CA00083FF20C08091E100877F8093E10082E074
:102CB00080937C03109278038091E1008E7F809353
:102CC000E1008091E2008E7F8093E2008091E2003B
:102CD00080618093E20042E060E080E00E94481260
:102CE0000E942E10FF91EF91BF91AF919F918F9114
:102CF0007F916F915F914F913F912F910F900FBEF8
:102D00000F901F9018950895CF9380917C0388238E
:102D1000A1F0C091E900CF709091EC00892F8170F3
:102D200090FD80E8C82B1092E9008091E80083FDB7
:102D30000E94DB13CF70C093E900CF910895909368
:102D40007D0280937C020895E0917C02F0917D02E7
:102D5000309721F00190F081E02D099480E00895F2
:102D6000EF92FF920F931F93CF93DF93E0917C023A
:102D7000F0917D023097B1F18C010280F381E02D5A
:102D800009958091720382FF2DC080FF04C087E403
:102D900097E00E94C305E80110E281E4E82E87E095
:102DA000F82E8091720380FF0BC088811F928F9351
:102DB000FF92EF920E945C060F900F900F900F9081
:102DC000115021961111EDCF8091720380FF0AC03E
:102DD0008FE397E0DF91CF911F910F91FF90EF90DC
:102DE0000C94C305DF91CF911F910F91FF90EF904D
:102DF0000895CF93DF9320917A0230917B022817B8
:102E0000390709F190937B0280937A02E0917C026A
:102E1000F0917D023097B9F0EC010680F781E02D4A
:102E200009958091720382FF0EC080FF0CC0DF9372
:102E3000CF9381E397E09F938F930E945C060F905E
:102E40000F900F900F90DF91CF910895CF93DF9364
:102E500020917802309179022817390709F190936F
:102E6000790280937802E0917C02F0917D023097A4
:102E7000B9F0EC010084F185E02D09958091720391
:102E800082FF0EC080FF0CC0DF93CF9381E297E0FA
:102E90009F938F930E945C060F900F900F900F905E
:102EA000DF91CF9108950C94FC170E948A230C9413
:102EB000510ABF92CF92DF92EF92FF920F931F932E
:102EC000CF93DF9300D000D01F92CDB7DEB70E9422
:102ED000760A0FE712E0F12C8F2D0E945E0AB82EC1
:102EE000F801C080C82639F4F3940F5F1F4FF0E15A
:102EF000FF12F2CF30C08091720381FD0E94FD1756
:102F0000D12CEE24E3948C2D8E21F9F0D982FA8213
:102F100091E08B2D8E2109F490E09B830E949323F6
:102F20008160782F9D838C8349815A816B818D814B
:102F30000E94331849815A816B817C818D810E9466
:102F40002B23F80180818E258083D394EE0CF8E04A
:102F5000DF12D9CFC9CF8FEF89838A831B820E946A
:102F600093238160782F9D838C8349815A816B8163
:102F70008D810E9433180E942A230E94A4169091EA
:102F80007E02891741F10E94A41680937E029091DF
:102F9000720392FF0EC090FF0CC01F928F9382E5C8
:102FA00097E09F938F930E945C060F900F900F9075
:102FB0000F9080917E020F900F900F900F900F90C6
:102FC000DF91CF911F910F91FF90EF90DF90CF9005
:102FD000BF900C943C230F900F900F900F900F9088
:102FE000DF91CF911F910F91FF90EF90DF90CF90E5
:102FF000BF9008950C946C0A0895EF92FF920F937E
:103000001F93CF93DF938BE697E00E94C305C0E048
:10301000D0E08CE2E82E81E0F82E0DE517E08C2F51
:103020000E945E0A0E941823FF92EF921F928F93D4
:10303000DF93CF931F930F930E945C0621968DB769
:103040009EB708960FB6F8949EBF0FBE8DBFC031D5
:10305000D10529F7DF91CF911F910F91FF90EF904C
:10306000089508950895CF93DF93CDB7DEB72B97DA
:103070000FB6F894DEBF0FBECDBF942F4F83252F20
:10308000588769877A878B874A855B85452B31F01E
:103090002F3F31F481E09F3F19F403C081E001C06C
:1030A00080E080FD07C04F81588569857A858B85D2
:1030B0000E942B23DE01119686E0FD0111928A9574
:1030C000E9F785E0FE01379601900D928A95E1F7C8
:1030D00049815A816B817C818D819E810E94261F4E
:1030E0002B960FB6F894DEBF0FBECDBFDF91CF9108
:1030F0000895CF93882309F465C0C82F8CEF8C0FF7
:10310000813A20F080E58C0F8E3248F48C2F0E949B
:103110006325811157C08C2F0E940E220CC080E2C3
:103120008C0F883058F4C77081E001C0880FCA95B1
:10313000EAF70E94B322CF910C94ED228BE58C0F1D
:10314000833078F4C53A29F0C63A31F083E890E04C
:1031500005C081E890E002C082E890E0CF910C9435
:10316000F91688E58C0F853168F5C83A89F0C93AB7
:1031700091F0CA3A99F0CB3AA1F0CC3AA9F0CD3A05
:10318000B1F0CE3AB9F0CF3AC1F080E090E017C08C
:1031900082EE90E014C089EE90E011C08AEE90E0DB
:1031A0000EC085EB90E00BC086EB90E008C083EB8F
:1031B00090E005C084EB90E002C087EB90E0CF91F7
:1031C0000C942617CF910895882349F19CEF980F0E
:1031D000913A20F090E5980F9E3218F40E945E22FA
:1031E0000DC090E2980F983058F4877091E001C0BC
:1031F000990F8A95EAF7892F0E94B9220C94ED2243
:103200009BE5980F933020F480E090E00C94F91641
:10321000885A853120F480E090E00C9426170895B8
:10322000882321F00E94B3220C94ED220895882374
:1032300021F00E94B9220C94ED2208950E94D3221D
:103240000E94A2220E94ED2280E090E00E94F916E6
:1032500080E090E00C9426170E94C3220C941E1963
:10326000CF92DF92EF92FF920F931F93CF93DF9352
:1032700000D000D01F92CDB7DEB76C010E943E2374
:103280008111EAC285E0F601DE01119601900D92EE
:103290008A95E1F7F601408151812381348121151E
:1032A000310531F05F3F31F481E04F3F19F403C045
:1032B00081E001C080E080FDCFC2F601F280E580B0
:1032C000E2948FE0E82249835A83FB82722F3D8388
:1032D0002C836F2D8D810E948A218C010E9489216F
:1032E0000E947920E12FE295EF708E2F90E0FC0193
:1032F000E45CFE4F0C94B625812F807F1F708823DD
:1033000011F01295107FFF2049F0112309F43BC200
:10331000812F0E94C6220E94ED2235C2802F0E947A
:10332000E418112309F498C2812F0E94CC220F9037
:103330000F900F900F900F90DF91CF911F910F91F1
:10334000FF90EF90DF90CF900C94ED22812F807F43
:103350001F70803211F01295107F002319F0013098
:1033600009F12BC0FF20A9F0EE2059F1F1E0812FE7
:10337000EF1228C00F900F900F900F900F90DF91D9
:10338000CF911F910F91FF90EF90DF90CF900C9411
:10339000D622EE2021F021E0E21609F45DC20E945F
:1033A000D9222DC0FF20E9F085E08E1508F454C223
:1033B0000E94B022812329F022C0FF20F1F0E11009
:1033C00015C0812F0F900F900F900F900F90DF91ED
:1033D000CF911F910F91FF90EF90DF90CF900C94C1
:1033E000101994E09E1508F437C209C0F6018581D2
:1033F00080FFC9C18F708583E4CFE110D7C1812FD1
:103400004AC1812F86958695837019F08130B9F075
:1034100023C2FF2019F0C801937002C080E090E041
:103420000F900F900F900F900F90DF91CF911F9101
:103430000F91FF90EF90DF90CF900C94F916FF2042
:1034400019F0C801937002C080E090E00F900F90D7
:103450000F900F900F90DF91CF911F910F91FF90E0
:10346000EF90DF90CF900C942617812F837009F096
:1034700070C0F110F1C1202F229526952770220FE0
:10348000220F602F6F70862F90E0A0E0B0E06C01FB
:103490007D01022E04C0CC0CDD1CEE1CFF1C0A9426
:1034A000D2F704FF12C08FE090E0A0E0B0E004C0CB
:1034B000880F991FAA1FBB1F2A95D2F7BC01CD0107
:1034C000609570958095909503C060E070E0CB01A9
:1034D0001695169513701230B1F040F56C297D29C0
:1034E0008E299F29113031F10F900F900F900F907E
:1034F0000F90DF91CF911F910F91FF90EF90DF9090
:10350000CF900C949E206C297D298E299F290F90A5
:103510000F900F900F900F90DF91CF911F910F910F
:10352000FF90EF90DF90CF900C94B8200E949E20E7
:10353000C701B6010F900F900F900F900F90DF9181
:10354000CF911F910F91FF90EF90DF90CF900C944F
:103550008420FF2019F0812F817001C08695882377
:1035600009F47AC1202F229526952770220F220F69
:10357000602F6F70862F90E0A0E0B0E06C017D01BD
:10358000022E04C0CC0CDD1CEE1CFF1C0A94D2F7EA
:1035900004FF12C08FE090E0A0E0B0E004C0880F0C
:1035A000991FAA1FBB1F2A95D2F7BC01CD016095B8
:1035B00070958095909503C060E070E0CB01169502
:1035C000169513701230B1F040F56C297D298E29C3
:1035D0009F29113031F10F900F900F900F900F90A5
:1035E000DF91CF911F910F91FF90EF90DF90CF90DF
:1035F0000C9465216C297D298E299F290F900F90AD
:103600000F900F900F90DF91CF911F910F91FF902E
:10361000EF90DF90CF900C9477210E946521C70135
:10362000B6010F900F900F900F900F90DF91CF91F8
:103630001F910F91FF90EF90DF90CF900C9453214A
:10364000003FC1F128F480E4800F803250F096C032
:10365000023F09F45EC008F449C0033F09F46CC09E
:103660008DC0F02FF071EF2E812F8F71FF2051F060
:103670000E94EC20802FEE2019F08295807FA2CE50
:103680008F70A0CE0E940D21802FEE2019F0829520
:10369000807F01C08F700F900F900F900F900F9050
:1036A000DF91CF911F910F91FF90EF90DF90CF901E
:1036B0000C941719FF20A9F024E02E1508F4CCC0B3
:1036C000812F8F710F900F900F900F900F90DF91BF
:1036D000CF911F910F91FF90EF90DF90CF900C94BE
:1036E000322185E08E1508F4B7C0EACFFF2099F0AB
:1036F000812F8F710F900F900F900F900F90DF918F
:10370000CF911F910F91FF90EF90DF90CF900C948D
:10371000EC20FF2069F3812F8F710F900F900F9095
:103720000F900F90DF91CF911F910F91FF90EF902D
:10373000DF90CF900C940D21FF2089F0812F8F71A5
:103740000F900F900F900F900F90DF91CF911F91DE
:103750000F91FF90EF90DF90CF900C94D7200F90B7
:103760000F900F900F900F90DF91CF911F910F91BD
:10377000FF90EF90DF90CF900C94D220FF2099F033
:10378000EE2009F4B5CF802F0F900F900F900F907F
:103790000F90DF91CF911F910F91FF90EF90DF90ED
:1037A000CF900C947918EE2009F4B5CF802F0F90AC
:1037B0000F900F900F900F90DF91CF911F910F916D
:1037C000FF90EF90DF90CF900C94E418412F4F7052
:1037D000602FC6010E94FE230F900F900F900F9054
:1037E0000F90DF91CF911F910F91FF90EF90DF909D
:1037F000CF900C94D41F01112FC0FF2069F10E94BB
:103800002C199FEFE0E7F2E09150E040F040E1F743
:1038100000C000000F900F900F900F900F90DF915D
:10382000CF911F910F91FF90EF90DF90CF900C946C
:10383000DF23412F4F70602FC6010F900F900F9024
:103840000F900F90DF91CF911F910F91FF90EF900C
:10385000DF90CF900C9401240F900F900F900F9059
:103860000F90DF91CF911F910F91FF90EF90DF901C
:10387000CF9008951F93CF93DF9300D000D01F9275
:10388000CDB7DEB7942F4983252F5A836B837C8372
:103890008D834C815D81452B31F02F3F31F481E0E8
:1038A0009F3F19F403C081E001C080E0182F117020
:1038B00080FD31C049815A816B817C818D810E945C
:1038C0008A21292F22952F702C3030F42A30A0F431
:1038D0002250223030F022C02C30C9F02F30B9F005
:1038E0001DC0853A28F48430C0F4823028F415C015
:1038F00090E2980F983088F0883E30F4803E68F46B
:103900008450813A58F409C0803F41F406C093FBCB
:10391000112710F903C010E001C011E0812F0F90B2
:103920000F900F900F900F90DF91CF911F910895FE
:10393000CF93DF9300D000D01F92CDB7DEB70F90AA
:103940000F900F900F900F90DF91CF910895CF932C
:10395000DF9300D000D000D0CDB7DEB726960FB6EB
:10396000F894DEBF0FBECDBFDF91CF9108951F93B6
:10397000CF93DF93C0918F0216E080919002C81719
:1039800099F0D0E01C9FF0011D9FF00D1124EF561F
:10399000FD4F4081518162817381848195810E94B4
:1039A000A71C2196C770E9CFDF91CF911F91089591
:1039B0004091C1025091C2026091C3027091C40251
:1039C0008091C5029091C6020C94A71C0F931F937F
:1039D000CF93DF938091C60282958F7009F05DC00E
:1039E0008091C302882309F458C080918F021091FE
:1039F00090026091C1027091C202C091C402D09144
:103A0000C50291E06F3F09F090E0292F06E0811791
:103A100009F443C0209721F07F3F21F030E003C03C
:103A200031E001C0322F90E030FD34C0089FF0013A
:103A3000099FF00D1124DF01AF56BD4F11963C9147
:103A40001197371327C03C91361324C012963C912E
:103A5000129731111FC013964D915C9114974C1B16
:103A60005D0B483C5105B0F48091C6028F708061B7
:103A70008093C602EA56FD4F80818F7080618083FB
:103A800081EC92E00E943019DF91CF911F910F914C
:103A90000C94B71C01968770BACFDF91CF911F911C
:103AA0000F9108959F92AF92BF92CF92DF92EF92C3
:103AB000FF920F931F93CF93DF93CDB7DEB761973C
:103AC0000FB6F894DEBF0FBECDBF8C0185E0F801C4
:103AD000DE011D9601900D928A95E1F7F801408173
:103AE0005181F280C380D4809091C1026091C20262
:103AF0002091C4023091C5022115310531F06F3F8C
:103B000031F481E09F3F19F403C081E001C080E0FF
:103B1000F82FF1709F2E80FD52C181ECA82E82E01B
:103B2000B82EE090C302F601E21BF30BEE2009F47D
:103B3000E8C08091C602E83CF10508F0A4C0282F37
:103B4000207F09F053C0561313C0491311C0EF2C46
:103B5000F1100EC08F7080618093C6020E94D81C45
:103B6000C5010E9430198091C602F80185835BC1AE
:103B7000C114D10431F05F3F31F481E04F3F19F4BB
:103B800003C081E001C080E080FD03C081E08F259B
:103B900002C080E090E0F82FF170EF2E80FF1CC093
:103BA00080918F022091900236E0821709F418C1AB
:103BB00090E0389FF001399FF00D1124EF56FD4F32
:103BC0006181561306C06081461303C06281F612FC
:103BD00003C001968770E9CFEF2CFF2009F423C1C1
:103BE0008091C60281608093C60262C0561306C0EF
:103BF000491304C0F11002C0F801A7C04D875E87C9
:103C0000FF867C2DD98AC88A6F2D89890E943A1C2B
:103C1000882399F1FF2089F12091C602822F829595
:103C20008F7090E0029774F08091C1029091C2026F
:103C300098878F831986DB86CA862C87CE010796E4
:103C40000E94301986E0F801A1ECB2E001900D92DB
:103C50008A95E1F70E94E61C0E94D81C11C05617F5
:103C600049F14D875E87FF867C2DD98AC88A6F2DE2
:103C700089890E943A1C81112CC0C8010E94301908
:103C8000EE24E394D0C0282F207F49F77C2DD98AD9
:103C9000C88A6F2D89890E94981C81EC92E00E944D
:103CA000301986E0F50111928A95E9F70E94D81C37
:103CB000E12CB9C04913D5CFF110D3CFF8018583DA
:103CC000C8010E94301986E0F50111928A95E9F742
:103CD000AAC0FF2091F22091C602822F82958F7098
:103CE00090E002970CF4AECF8091C1029091C20295
:103CF0009A8389831B82DD82CC822E83CE0101963A
:103D00009FCFE83CF10508F04BC0EF2CFF2009F4F1
:103D1000B4CF561330C049132EC02091C60220FDE7
:103D200021C0822F82958F70482F50E04115510598
:103D3000C9F0F80125834F30510541F08F5F982F6E
:103D40009295907F822F8F70892B8583C8010E9466
:103D5000301986E0F801A1ECB2E001900D928A954D
:103D6000E1F72AC086E0F801A1ECB2E001900D92E3
:103D70008A95E1F758C04D875E87FF867C2DD98AEA
:103D8000C88A6F2D89890E943A1C81115BCF80916E
:103D9000C60281608093C602C8010E94301943C0E8
:103DA0007C2DD98AC88A6F2D89890E94981C86E04B
:103DB000F50111928A95E9F70E94D81C34C0FF20C2
:103DC00009F45BCF4D875E87FF867C2DD98AC88A30
:103DD0006F2D89890E943A1C882309F44ECF32CF77
:103DE0007C2DD98AC88A6F2D89890E948A21292F22
:103DF00022952F70223028F49F7039F0811105C070
:103E00000BC0243028F49F7049F4805E883020F085
:103E1000C8010E9430199E2CE92C05C0F80195813B
:103E2000907F99F7F9CF8E2D61960FB6F894DEBF8B
:103E30000FBECDBFDF91CF911F910F91FF90EF90FB
:103E4000DF90CF90BF90AF909F9008951F93CF9336
:103E5000DF93CDB7DEB72C970FB6F894DEBF0FBE59
:103E6000CDBF4F83588769877A878B879C87CE0120
:103E700007960E94521D8823D1F09F8188852A854C
:103E80003B85232B31F08F3F31F481E09F3F19F4C4
:103E900003C081E001C080E080FD47C04F815885AC
:103EA00069857A858B859C850E94A71C3EC086E02B
:103EB000FE013796DE01119601900D928A95E1F789
:103EC000FF81E8856A857B856115710531F0EF3FDB
:103ED00031F481E0FF3F19F403C081E001C080E0CC
:103EE00080FD23C02091900230E0C90101968770C7
:103EF000992740918F0250E084179507F1F1F983DB
:103F0000EA837D836C8396E0929FD001939FB00DEE
:103F10001124AF56BD4FFE01319601900D929A9536
:103F2000E1F7809390020E94B71C16E080918F0207
:103F300090919002891771F1189FC00111248F563A
:103F40009D4F0E94521D882329F1E0918F021E9FF0
:103F5000F0011124EF56FD4F408151816281738140
:103F6000848195810E94A71C80918F0290E0019628
:103F70008770992780938F02D9CF0E942C191092B5
:103F8000900210928F02E1ECF2E086E0DF011D92D8
:103F90008A95E9F72C960FB6F894DEBF0FBECDBF19
:103FA000DF91CF911F910895DF92EF92FF920F93CF
:103FB0001F93CF93DF93FC01892B09F488C0E12C78
:103FC000F12CDD24D394EF0121968491853709F4F7
:103FD00060C058F4843708F04EC0843008F068C0E0
:103FE0008130D1F0823071F172C0883709F45BC042
:103FF00050F4863709F453C0873709F068C08E2D16
:104000000E94C02252C09CE7980F903708F05FC012
:104010008F770E94E4184EC08F010E5F1F4FFE0184
:10402000849190E2980F983050F48770FD2D01C074
:10403000FF0F8A95EAF78F2F0E94C62215C00E94B3
:10404000791814C08F010E5F1F4FFE01849190E21A
:10405000980F983068F48770FD2D01C0FF0F8A9586
:10406000EAF78F2F0E94CC220E94ED22E80122C0A5
:104070000E94E418FBCFCF010296FE01C491CC232D
:1040800061F0EFE9FFE03197F1F700C00000C150A7
:10409000F6CFCF010296FE01F490EC010BC00E9416
:1040A000B022E82E07C00E94C3220E94ED2202C067
:1040B0000E9479188F2D882341F0EFE9FFE03197B6
:1040C000F1F700C000008150F6CFFE017CCFDF91F8
:1040D000CF911F910F91FF90EF90DF900895609323
:1040E0004703709348038093490390934A030C94C9
:1040F0003B23089560934B0370934C0380934D03CF
:1041000090934E030C943A230F931F9300914B030B
:1041100010914C0320914D0330914E03602B712B75
:10412000822B932B60934B0370934C0380934D032E
:1041300090934E031F910F910C943A230F931F936A
:1041400000914B0310914C0320914D0330914E038D
:10415000602371238223932360934B0370934C035A
:1041600080934D0390934E031F910F910C943A232B
:104170000F931F9300914B0310914C0320914D031B
:1041800030914E03602771278227932760934B035A
:1041900070934C0380934D0390934E031F910F91A6
:1041A0000C943A2360E070E0CB010C946F200F93E5
:1041B0001F9341E050E060E070E08A019B0104C081
:1041C000000F111F221F331F8A95D2F7C901B801B2
:1041D0001F910F910C946F200F931F9341E050E0BB
:1041E00060E070E004C0440F551F661F771F8A957A
:1041F000D2F78091470390914803A0914903B09171
:104200004A038A019B01082B192B2A2B3B2BC9013E
:10421000B8011F910F910C946F200F931F9341E0F1
:1042200050E060E070E004C0440F551F661F771F28
:104230008A95D2F740955095609570958091470387
:1042400090914803A0914903B0914A038A019B01D0
:10425000082319232A233B23C901B8011F910F9179
:104260000C946F200F931F9341E050E060E070E0EA
:1042700004C0440F551F661F771F8A95D2F780919F
:10428000470390914803A0914903B0914A038A01E2
:104290009B01082719272A273B27C901B8011F912D
:1042A0000F910C946F200F931F930091470310916F
:1042B00048032091490330914A03602B712B822BD4
:1042C000932B1F910F910C946F200F931F930091CC
:1042D0004703109148032091490330914A0360231A
:1042E0007123822393231F910F910C946F200F93BE
:1042F0001F93009147031091480320914903309187
:104300004A0360277127822793271F910F910C94EE
:104310006F2008958F929F92AF92BF92DF92EF929B
:10432000FF920F931F93CF93DF9300D000D01F9283
:10433000CDB7DEB76B837C838D838A018C819D81B1
:10434000892B31F01F3F31F481E04F3F19F403C056
:1043500081E001C080E080FF03C080E090E04DC0BC
:104360008B818823D1F18090470390904803A090DF
:104370004903B0904A0380914B0390914C03A09164
:104380004D03B0914E03882A992AAA2ABB2A8FE1AD
:10439000E82EF12CD501C4010E2C04C0B695A795CA
:1043A000979587950A94D2F780FD06C081E0E81AB8
:1043B000F10880F7D12C07C0DE2CB8018E2D0E94A9
:1043C0006506019799F388E0189FF0011124E953DD
:1043D000FD4FE00FF11DD08209C088E0189FF00169
:1043E0001124E953FD4FE00FF11DD08009831A839A
:1043F00069817A818D2D0E9465060F900F900F9034
:104400000F900F90DF91CF911F910F91FF90EF9040
:10441000DF90BF90AF909F908F900895909114017E
:10442000992379F190911501992359F1982F969537
:10443000969596959F31A1F0E0911601F0911701A4
:10444000E90FF11D877021E030E0A90102C0440F9F
:10445000551F8A95E2F7CA019181892B81830895BE
:104460009091720390FF29C01F928F9387E997E084
:104470009F938F930E945C060F900F900F900F9068
:1044800008952091160130911701F90132969FEF9E
:1044900040E05191851789F09F3F19F4511101C0F7
:1044A000942F4F5F4E31A9F79F3F39F0F901E90F83
:1044B000F11D97FDFA958283089508959091140156
:1044C000992381F190911501992361F1982F969587
:1044D000969596959F31A9F0E0911601F0911701FC
:1044E000E90FF11D877021E030E0A90102C0440FFF
:1044F000551F8A95E2F7CA018095918189238183AE
:1045000008959091720390FF1CC01F928F9389E7CA
:1045100097E09F938F930E945C060F900F900F90EF
:104520000F900895E0911601F09117019F01225E0E
:104530003F4F9281891301C012823196E217F3072F
:10454000C1F7089581E090E0E0911601F091170124
:10455000E80FF91F1082019680329105A9F708959E
:1045600080917103089590917103892B8093710359
:104570000895809590917103892380937103089524
:1045800080937103089510927103089590917003C0
:10459000892B8093700308958095909170038923EF
:1045A00080937003089510927003089580934F03D1
:1045B000089510924F03089580911601909117016C
:1045C000FC0131969C01205E3F4F80E0919191115A
:1045D0008F5FE217F307D1F70895E0911601F0918C
:1045E0001701809171038083E0911601F09117010A
:1045F000908180917003892B808380914F03882361
:1046000061F0E0911601F09117019081892B808370
:104610000E94DC22811110924F038091160190912B
:1046200017010C94B01690933501809334010895CE
:104630008295982F937344E0949F900111248C7C71
:1046400086958695282B822F8575880F2A7A269540
:10465000822B08950895CF93DF9300D000D01F924E
:10466000CDB7DEB70F900F900F900F900F90DF91A6
:10467000CF910895089508950C94FA1780E0089555
:1046800083B7817F8C6083BF83B7816083BF789459
:10469000889583B78E7F83BF0895CF930E9431188A
:1046A0000E94760A0E943218C0E08C2F0E945E0A97
:1046B000811104C0CF5FC031C1F701C081E0CF914B
:1046C00008950E94640A0C942C191F920F920FB641
:1046D0000F9211248F939F93AF93BF938091730395
:1046E00090917403A0917503B09176034196A11D3A
:1046F000B11D8093730390937403A0937503B093DB
:104700007603BF91AF919F918F910F900FBE0F9045
:104710001F90189582E084BD93E095BD9AEF97BDF8
:1047200080936E0008952FB7F89480917303909151
:104730007403A0917503B09176032FBF08952FB72E
:10474000F894609173037091740380917503909154
:1047500076032FBF08959C014FB7F894809173039F
:1047600090917403A0917503B09176034FBF821BA3
:10477000930B08951F920F920FB60F9211248F93EF
:104780009F93AF93BF938091730390917403A09113
:104790007503B09176030196A11DB11D809373033B
:1047A00090937403A0937503B0937603BF91AF9178
:1047B0009F918F910F900FBE0F901F9018950E94A0
:1047C0003B15F89487E797E79093010880930008DA
:1047D00087E090EBDC018093850390938603A093A0
:1047E0008703B09388039CE088E10FB6F894A895FE
:1047F000809360000FBE90936000FFCF80E090E058
:1048000008950895CF93C82F1F928F938BEB97E055
:104810009F938F930E945C0681E090E0A0E0B0E05F
:10482000BC01CD0104C0660F771F881F991FCA9570
:10483000D2F70E947A200F900F900F900F90CF9197
:104840000C942C19CF938732A8F58E3108F02BC128
:10485000803109F49FC0F8F4873009F464C0A8F4EB
:10486000863009F024C180917203817F8E7F80930E
:10487000720380EC97E00E94C30583EA9AE00E94ED
:10488000C30581E0809377034CC08B30F1F18E300B
:1048900009F46CC00CC1863109F4B0C020F4813138
:1048A00009F4EDC004C1893109F491C08B3109F4D8
:1048B00049C0FDC0883349F150F4893209F4F1C090
:1048C000853309F4EEC0873209F0F1C0EAC08334C1
:1048D00009F4E7C028F48A3308F4E9C08953E4C036
:1048E000883409F0E4C00E942C1982E99AE00E9401
:1048F000C3052FEF83ED90E3215080409040E1F716
:1049000000C000000E94DF230CC08BED97E05CC06C
:1049100089E79AE00E94C3058091720381608093C9
:104920007203C1E0C9C080917203C82FC17080FFBB
:10493000EFCF85E89AE00E94C30580917203817FE2
:104940008E7F3DC09091720391FBCC27C0F981E02E
:10495000C827892FC0FB81F980937203CC2319F0FB
:104960008CE69AE027C08EE59AE02EC09091720303
:1049700092FBCC27C0F981E0C827892FC0FB82F9C0
:1049800080937203CC2319F08FE49AE013C08FE375
:104990009AE01AC09091720393FBCC27C0F981E092
:1049A000C827892FC0FB83F980937203CC2351F071
:1049B00083E39AE00E94C305809172038160809333
:1049C00072037AC086E29AE00E94C305AACF87E10B
:1049D0009AE00E94C30581EF99E00E94C30589EA2D
:1049E00099E00E94C30580E899E00E94C30584E332
:1049F00099E00E94C30589E099E0E6CF8BEF98E04B
:104A00000E94C3050E94A4161F928F9381EE98E026
:104A10009F938F930E945C06809114011F928F9345
:104A20008AEC98E09F938F930E945C0680917702B6
:104A30001F928F9387EB98E09F938F930E945C0661
:104A4000809115011F928F9384EA98E09F938F9332
:104A50000E945C060E949F239F938F937F936F9386
:104A60008DE898E09F938F930E945C068DB79EB768
:104A700046960FB6F8949EBF0FBE8DBF52CF0E94D0
:104A80002C19C091150181E0C827C0931501CC23D2
:104A900029F083E898E00E94C3050EC088E798E0FB
:104AA00093CF80E001C08D510E9402243ACF86E767
:104AB00098E00E94C305C0E08C2FCF91089580E05C
:104AC00008950C945F25CF93C82F80917703882396
:104AD00019F0813059F042C0E0911601F0911701B0
:104AE0008081823261F08434D9F509C0E0911601E9
:104AF000F09117018081823211F0843461F48C2F9F
:104B00000E946125811104C08C2F0E94222424C0A0
:104B100081E090E021C08C2F0E945F2581111BC095
:104B2000C43189F018F4CB3029F010C0C93259F0E3
:104B3000C83361F480EC97E00E94C30587EB97E0EF
:104B40000E94C30508C0109277030CC085EB97E064
:104B50000E94C30507C081E0817006C010927703F0
:104B600080E002C080E0F8CFCF910895EE0FFF1FE4
:0C4B70000590F491E02D0994F894FFCF1B
:104B7C000080FFFF0556010000FF5B0EC80E5E0EA5
:104B8C00930E5F0E0101500340362239E106AB064D
:104B9C0089065006DC05F5050E062E0600000800F9
:044BAC0004000200FF
:106800008800EA44E944E244040005000600070069
:10681000080009000A000B000C000D000E000F001C
:1068200010001100120013001400150016001700CC
:10683000180019001A001B001C001D001E001F007C
:10684000200021002200230024002500260027002C
:10685000280029002A002B002C002D002E002F00DC
:10686000300031003200330034003500360037008C
:10687000380039003A003B003C003D003E003F003C
:1068800040004100420043004400450046004700EC
:10689000480049004A004B004C004D004E004F009C
:1068A000500051005200530054005500560057004C
:1068B000580059005A005B005C005D005E005F00FC
:1068C0006000610062006300640065A185006700EC
:1068D000680069006A006B006C006D006E006F005C
:1068E0007000710072007300890087008A008B00BD
:1068F000E000E100E200E300E400E500E600E7007C
:106900000100010001000100EA4401000100E2442D
:106910000100010001000100460001004A004B0097
:10692000010001004700480001000100E9440100A6
:106930000100010001000100010001003A003B00DC
:106940003C003D003E003F0040004100420043004B
:10695000010035004C0039000100440045005200A0
:1069600049000100010050004F0029004D004E0079
:1069700051000100010001000100010001000100BF
:1069800001000100010001000100010001000100FF
:1069900001000100010001000100010001004D00A3
:1069A0004A004E004B0001000100010001000100FF
:1069B00001000100010001000100010001000100CF
:1069C00001000100010001000100010001000100BF
:1069D00001000100010001000100010001000100AF
:1069E0000100010001000100490001000100010057
:1069F000010001000100010001000100010001008F
:00000001FF
